:100000000C9462000C948A000C948A000C94790180
:100010000C94A6010C94D3010C948A000C948A00D1
:100020000C948A000C948A000C948A000C948A0028
:100030000C948A000C947C0B0C948A000C948A001B
:100040000C94A30B0C948A000C948A000C948A00E4
:100050000C948A000C948A000C948A000C948A00F8
:100060000C948A000C948A000000000024002700F1
:100070002A0000000000250028002B0000000000DE
:1000800023002600290004040404040404040202DA
:100090000202020203030303030301020408102007
:1000A0004080010204081020010204081020000012
:1000B0000007000201000003040600000000000029
:1000C0000000000211241FBECFEFD8E0DEBFCDBF7D
:1000D00012E0A0E0B1E0EAEDF5E202C005900D9279
:1000E000A636B107D9F712E0A6E6B2E001C01D922C
:1000F000A73DB107E1F710E0C4ECD0E004C02297BF
:10010000FE010E94E712C23CD107C9F70E946B0EA4
:100110000C94EB120C940000CF93DF93EC01DB0105
:1001200012962C93129711965C934E93EA81FB8161
:10013000808113969C911397892B808312968C91C2
:100140001297833011F0813031F48D8113969C9198
:100150001397892B8D8312968C9112978150823040
:1001600028F48E8113969C91892B8E838091680050
:100170009C81892B80936800DF91CF910895CF9364
:10018000DF93282F30E0F901EA57FF4F849188234D
:1001900009F44FC0833051F0843059F0823019F4A3
:1001A000A9E6B2E008C0A0E0B0E005C0A3E7B2E075
:1001B00002C0ADE7B2E026563F4FF9019491189680
:1001C000CD91DC91199733C08B81891769F52FB7D1
:1001D000F8941296ED91FC91139780819095982355
:1001E00090831296ED91FC9113978081882349F4B6
:1001F0009091680014968C91149780958923809330
:10020000680015969C9115978B818095892315968A
:100210008C93159716969C9116978B8180958923C0
:1002200016968C932FBF05C00D80DE81C02D2097C0
:1002300059F6DF91CF910895EF92FF920F931F939C
:10024000CF93DF938C0150916602D80117962C91C1
:10025000179715964C9115979091660216963C91BA
:10026000169780916602809583239423892B2527F6
:1002700082239091660217969C9317971896CD91BA
:10028000DC911997E82EFF241CC08B81282F30E0C9
:10029000C70182239323892B89F08091660240E075
:1002A00090E082239323892B09F041E04093680278
:1002B0008C8180936702E881F98109950D80DE8148
:1002C000C02D209711F78BB3F8019481892351F049
:1002D0008BB3892B8BBB0190F081E02D80818093C3
:1002E0006602B1CFDF91CF911F910F91FF90EF90F8
:1002F00008951F920F920FB60F9211242F933F93E0
:100300004F935F936F937F938F939F93AF93BF931D
:10031000EF93FF93E0916902F0916A0280818093EC
:10032000660289E692E00E941C01FF91EF91BF9165
:10033000AF919F918F917F916F915F914F913F917D
:100340002F910F900FBE0F901F9018951F920F9234
:100350000FB60F9211242F933F934F935F936F9398
:100360007F938F939F93AF93BF93EF93FF93E0910E
:100370007302F091740280818093660283E792E0B9
:100380000E941C01FF91EF91BF91AF919F918F91BE
:100390007F916F915F914F913F912F910F900FBE81
:1003A0000F901F9018951F920F920FB60F92112465
:1003B0002F933F934F935F936F937F938F939F936D
:1003C000AF93BF93EF93FF93E0917D02F0917E0294
:1003D0008081809366028DE792E00E941C01FF916C
:1003E000EF91BF91AF919F918F917F916F915F91AD
:1003F0004F913F912F910F900FBE0F901F90189526
:10040000CF92EF920F93E0E8F0E085919491909372
:100410006A02809369028BE690E090936C0280936D
:100420006B0281E080936D0210926E0210926F0257
:100430001092720210927102E2E8F0E085919491BC
:1004400090937402809373028CE690E0909376020E
:100450008093750282E08093770210927802109266
:10046000790210927C0210927B02E4E8F0E0859120
:10047000949190937E0280937D028DE690E090931C
:10048000800280937F0284E0809381021092820236
:100490001092830210928602109285028FEA92E0F7
:1004A00068E049E024E005E056E0E52E37E0C32EA1
:1004B0000E943E0B0F91EF90CF9008958EE48093B1
:1004C0007C0062E070E080E090E00E94EB0B8091A5
:1004D0007A00806480937A0080917A0086FDFCCF58
:1004E0008091780060917900362F20E090E0282BF1
:1004F000392B442737FD4095542F6CEC74EA81E189
:1005000090E00E94CA12CA01B9010E9411116093C1
:10051000A7027093A8028093A9029093AA0208955B
:10052000EF92FF920F931F9388EC80937C0062E020
:1005300070E080E090E00E94EB0B80917A00806494
:1005400080937A0080917A0086FDFCCF209178001C
:1005500030E040E050E0E09179007E2F60E08827B5
:1005600077FD8095982F622B732B842B952B23E39B
:1005700034E040E050E00E948912675E7C40824097
:10058000904020E137E240E050E00E94CA12CA01E8
:10059000B9010E9411117B018C0160938702709355
:1005A00088028093890290938A0220E030E040E143
:1005B00051E40E94C11120E030E040EA50E40E9482
:1005C000761020E030E040E052E40E940E1060938C
:1005D0008B0270938C0280938D0290938E02C801DF
:1005E000B70123E333E948E853E40E94761020E0A2
:1005F00030E040E85FE30E940E100E94281220E0E5
:1006000030EC45EA53E40E94C1117B018C0120E0EB
:1006100030E04AEA53E40E947610609397027093A8
:1006200098028093990290939A02E092A302F0922A
:10063000A4020093A5021093A6021F910F91FF90B0
:10064000EF900895EF92FF920F931F930FEA12E03D
:10065000C80160E040E00E941509C80160E071E057
:100660000E94830FC8016AED0E943409C80163E04B
:1006700071E00E94830FC8016AED0E943409C8012D
:1006800065E071E00E94830FC8016AED0E943409A1
:100690006FE0E62E61E0F62EC801B7010E94830FDD
:1006A000C8016AED0E943409C80161E171E00E944D
:1006B000830FC80160E041E00E941509C80165E1AF
:1006C00071E00E94830FC80166E00E943409C801EE
:1006D0006CE171E00E94830FC8016AED0E94340949
:1006E000C8016EE171E00E94830FC8016AED0E94AB
:1006F0003409C801B7010E94830FC8016AED0E9446
:100700003409C80161E271E00E94830FC80160E012
:1007100042E00E941509C80168E271E00E94830F5F
:10072000C80166E00E943409C80161E371E00E94DB
:10073000830FC8016AED0E943409C80168E371E0C3
:100740000E94830F64EC79E080E090E00E94EB0B64
:10075000C8010E946F09C80160E041E00E941509CC
:10076000C8016DE371E00E94830FC80160E042E0C0
:100770000E941509C80162E571E00E94830F64ECD4
:1007800079E080E090E00E94EB0BC8010E946F09C5
:100790001F910F91FF90EF90089582E160E00E9419
:1007A000280D089581E160E00E94280D089582E1FE
:1007B00061E00E94280D08956F927F928F929F9220
:1007C000AF92BF92CF92DF92EF92FF920F931F935F
:1007D0000E94D7038AE060E00E94280D82E090E04A
:1007E0000E94440C8AE061E00E94280D8AE090E0BB
:1007F0000E94440C8AE060E00E94280D83E161E0E1
:1008000020E432E44FE050E00E94CF0D0E940F112F
:100810007B018C0160938F02709390028093910210
:100820009093920260909702709098028090990243
:1008300090909A0223E938E14BEE51E40E94761041
:1008400020E030E040E05FE30E94C111A401930189
:100850000E94C1115B016C0160939B0270939C022A
:1008600080939D0290939E02C801B70120E030E082
:1008700044E952E40E94761020E030E040E05FE37B
:100880000E94C111A40193010E94C11160939F02B3
:100890007093A0028093A1029093A202C601B501B9
:1008A00020E030E040E050E00E947210882321F404
:1008B00081E08093AE0202C01092AE021F910F91B0
:1008C000FF90EF90DF90CF90BF90AF909F908F9070
:1008D0007F906F9008952F923F924F925F926F9208
:1008E0007F928F929F92AF92BF92CF92DF92EF92C0
:1008F000FF920F931F93DF93CF9300D000D0CDB71B
:10090000DEB71B012C015C834B8320E030E040E02C
:1009100050E00E94721088232CF420E030E040E088
:100920005FEB04C020E030E040E05FE300E010E077
:100930000CC0CA01B90120E030E040E251E40E945D
:1009400076109B01AC010F5F1F4F8B819C810817B4
:1009500019077CF3C201B1010E940E105B016C010A
:10096000C201B10120E030E040E050E00E9472108E
:10097000882324F4D7FAD094D7F8D0940F2EFDEC26
:100980006F2EFCEC7F2EFCEC8F2EFDE39F2EF02DC6
:100990001A82198207C0E981FA813196FA83E983C4
:1009A00037014801C401B30120E030E040E251E4E6
:1009B0000E94C1117B018C01A60195010E94721059
:1009C00018164CF7C201B10120E030E040E050E0E1
:1009D0000E94721088232CF48FEA92E06DE20E944C
:1009E000A80E89819A81892B41F48FEA92E060E018
:1009F00070E04AE050E00E94700F4424552433C058
:100A0000C601B501A40193010E9476100E94DE1078
:100A10009B01AC017B018FEA92E0B9014AE050E012
:100A20000E94700F0027F7FC0095102FC801B70136
:100A30000E941111A40193010E94C1119B01AC01FC
:100A4000C601B5010E940D105B016C01C401B30128
:100A500020E030E040E251E40E9476103B014C017E
:100A60000894411C511CE981FA814E165F0644F23C
:100A70008B819C8118161906ACF58FEA92E06EE224
:100A80000E94A80E88249924C601B50120E030E018
:100A900040E251E40E94C1115B016C010E94DE1032
:100AA0009B01AC017B018FEA92E0B9014AE050E082
:100AB0000E94700F0027F7FC0095102FC801B701A6
:100AC0000E9411119B01AC01C601B5010E940D10DD
:100AD0005B016C010894811C911CEB81FC818E16DA
:100AE0009F0694F20F900F900F900F90CF91DF918F
:100AF0001F910F91FF90EF90DF90CF90BF90AF903C
:100B00009F908F907F906F905F904F903F902F902D
:100B10000895EF92FF920F931F931092AD021092DF
:100B2000AC020E9490020E945E020FEA12E0C8012D
:100B30000E946F09C80167E671E00E94830F60910F
:100B4000A7027091A8028091A9029091AA0220E0C8
:100B500030E04AE754E40E94761042E050E00E9400
:100B60006B04C8016DE671E00E94830FC80160E06C
:100B700041E00E941509C80160E771E00E94830FFF
:100B800060918702709188028091890290918A0217
:100B900041E050E00E946B0475E7E72E71E0F72E0C
:100BA000C801B7010E94830FC80162EB0E9434099B
:100BB000C80167E771E00E94830FC80160E042E06E
:100BC0000E941509C80169E771E00E94830F6091D6
:100BD0008B0270918C0280918D0290918E0241E087
:100BE00050E00E946B04C801B7010E94830FC80146
:100BF00062EB0E943409C8016EE771E00E94830F26
:100C0000C80160E043E00E941509C80160E871E096
:100C10000E94830F6091A3027091A4028091A502AB
:100C20009091A60242E050E00E946B04C80165E882
:100C300071E00E94830F68E873E180E090E00E9419
:100C4000EB0B1F910F91FF90EF90089581E161E010
:100C50000E94280D8FEA92E064E144E020E00E94C7
:100C600077090895882349F48FEA92E00E940A09DF
:100C70000E94D2030E94CD0308950E9426060E947E
:100C8000D703089583B78E7F83BF789481E00E9455
:100C9000320682E00E94BF00089580E00E947C0D31
:100CA000892B71F00E94420628E088E190E00FB69F
:100CB000F894A895809360000FBE20936000FFCF4A
:100CC00008950F931F938EE062E00E94E90C8FE07D
:100CD00062E00E94E90C82E062E00E94E90C80E19F
:100CE00062E00E94E90C83E160E00E94E90C8AE086
:100CF00061E00E94E90C81E161E00E94E90C82E17F
:100D000061E00E94E90C82E00E94BF000E9426067A
:100D10000E94D7030FEA12E0C80160E04AEF51E0F9
:100D20000E943F09C80161E042E052E00E943F0991
:100D3000C80162E04AE052E00E943F09C80163E056
:100D400042E152E00E943F09C80164E04AE152E0FA
:100D50000E943F09C80165E042E252E00E943F095B
:100D6000C80166E04AE252E00E943F09C80167E01C
:100D700042E352E00E943F09C8010E946F090E94AD
:100D800022031F910F910895CF92DF92EF92FF926D
:100D90000F931F93CF93DF938C01F62E6A01E22EFF
:100DA000FC01C085D185209789F08C818F1541F495
:100DB000C801BE01A6012E2D0E948C0080E03CC01F
:100DC0008D819E81009731F0EC01EFCF80E090E0C3
:100DD0009C01E90187E090E00E947B0EDC01119606
:100DE0001C921E9212961C921297009711F48FEF8C
:100DF00023C01496FC9214971296EC9212971696B2
:100E00001C921E921597EF2DF0E0E656FF4FE491ED
:100E10001396EC931397F80180859185892B19F42B
:100E2000B187A08702C0BE83AD83C801BD01A60102
:100E30002E2D0E948C0081E0DF91CF911F910F91A8
:100E4000FF90EF90DF90CF900895582F9B01742F63
:100E5000E82FF0E0EA57FF4F8491882311F1211524
:100E60003105F9F0833051F0843059F0823019F4B3
:100E7000A9E6B2E008C0A0E0B0E005C0A3E7B2E098
:100E800002C0ADE7B2E0ED91FC9111978081179619
:100E90008C931797CD01652FA901272F0E94C406B7
:100EA00008958FEF0895FF920F931F93FF24F394FB
:100EB000F092AB020FEA12E0C8010E946F09C8016C
:100EC0006AE871E00E94830FC8016AED0E9434094C
:100ED000C80163E071E00E94830FC8016AED0E94BF
:100EE0003409C8016DE871E00E94830FC80166ED06
:100EF0000E943409C80163E971E00E94830FC801B0
:100F00006AED0E943409C80166E971E00E94830F0E
:100F1000C8016AED0E943409C80169E971E00E94C4
:100F2000830F68EB7BE080E090E00E94EB0B0E9477
:100F3000D2030E94CD03EAE7F0E01081108282E044
:100F400080936900FDBA80E00E94320682E06DE481
:100F500076E040E050E00E94250783B7817F8460FF
:100F600083BFF89483B7816083BF85B7806685BFF0
:100F70008F7D85BF7894889583B78E7F83BF1093CC
:100F80007A001F910F91FF9008950E94DC036093F7
:100F900093027093940280939502909396020E941C
:100FA0005E020E9490028091AE02882309F050C038
:100FB0008FEA92E060E040E00E94150960919B0298
:100FC00070919C0280919D0290919E0242E050E0BF
:100FD0000E946B048FEA92E06CE971E00E94830F3B
:100FE0008FEA92E06AED0E9434098FEA92E063EAA8
:100FF00071E00E94830F8FEA92E060E041E00E947E
:10100000150960919F027091A0028091A1029091B8
:10101000A20242E050E00E946B048FEA92E06CEA88
:1010200071E00E94830F8FEA92E06AED0E9434091A
:101030008FEA92E061EB71E00E94830F8FEA92E009
:101040006AED0E9434098FEA92E061E271E042C0E9
:101050008FEA92E060E040E00E9415098FEA92E09A
:1010600063EB71E00E94830F8FEA92E06AED0E94C9
:1010700034098FEA92E06CEB71E00E94830F8FEAF3
:1010800092E06AED0E9434098FEA92E068E371E031
:101090000E94830F8FEA92E060E041E00E94150910
:1010A0008FEA92E063EC71E00E94830F8FEA92E096
:1010B0006AED0E9434098FEA92E06BEC71E00E94C5
:1010C000830F8FEA92E064E00E9434098FEA92E095
:1010D0006FEC71E00E94830F8FEA92E060E042E0E3
:1010E0000E9415098FEA92E068ED71E00E94830F7B
:1010F0008FEA92E060E043E00E9415098FEA92E0F7
:101100006DEE71E00E94830F8FEA92E067E00E942B
:1011100034098FEA92E065E771E00E94830F6091E5
:10112000A7027091A8028091A9029091AA0220E0E2
:1011300030E04AE754E40E94761042E050E00E941A
:101140006B048FEA92E06DE671E00E94830F64EF1A
:1011500071E080E090E00E94EB0B8091AC029091F6
:10116000AD0201969093AD028093AC0280E10E94A3
:101170007C0D892B31F08091AC029091AD02889763
:1011800034F01092AD021092AC020E9453078EE030
:101190000E947C0D892B11F40E9489050895089501
:1011A0000895FC011382128282E492E0918380838D
:1011B0000895FC01A081B18118962D913C91199759
:1011C0006FEFF90109950895FC01A081B18118968E
:1011D0002D913C91199760E0F90109950895DC0182
:1011E000ED91FC910284F385E02D40E0099508958E
:1011F000FC016581862F846085836C60CF010E942D
:10120000EF080895FC0165816B7F658368600E942B
:10121000EF0808950F931F938C010E94E408C80102
:101220000E9402091F910F910895DC0117969C916D
:101230001797491710F0492F415018968C9118971D
:10124000803139F4943029F4E42FF0E0E25BFD4F73
:1012500004C0E42FF0E0EE5AFD4F8081680F606813
:10126000CD010E94EF080895DC01ED91FC9102840C
:10127000F385E02D41E0099581E090E00895EF923B
:10128000FF920F931F93CF93DF938C017A016770C6
:10129000660F660F660F60640E94EF088EE190E0B3
:1012A0000E94440CC0E0D0E0D801ED91FC91D70140
:1012B000AC0FBD1F0190F081E02DC8016C91099524
:1012C00088E290E00E94440C2196C830D10561F775
:1012D000DF91CF911F910F91FF90EF90089561E002
:1012E0000E94EF0880ED97E00E94440C0895CF9390
:1012F000DF93EC01423018F08C8188608C834F833F
:101300006887222329F0413019F48C8184608C8312
:1013100064E670E080E090E00E94EB0B6C8164FD7D
:1013200031C0E881F9810284F385E02DCE0163E0CC
:1013300042E0099584E991E10E94440CE881F98139
:101340000284F385E02DCE0163E042E0099584E953
:1013500091E10E94440CE881F9810284F385E02D3B
:10136000CE0163E042E0099586E990E00E94440CDA
:10137000E881F9810284F385E02DCE0162E042E04C
:10138000099516C06062CE010E94EF0884E991E1E0
:101390000E94440C6C816062CE010E94EF0886E9D5
:1013A00090E00E94440C6C816062CE010E94EF08C4
:1013B0006C816062CE010E94EF0884E08D83CE01D3
:1013C0000E94F808CE010E946F0982E08E83CE0150
:1013D00066E00E94EF08CE010E94D908DF91CF910C
:1013E00008950F931F938C01FC01858561E00E9495
:1013F000280DF801858560E00E94280D1F910F914E
:101400000895BF92CF92DF92EF92FF920F931F93B6
:10141000CF93DF93D82EC92EB42E282F392FC90190
:101420008C01C0E0D0E0E62EFF240DC0B7010C2EE9
:1014300002C0759567950A94E2F76170F801858599
:101440000E94280D21960F5F1F4FCB1578F38D2D2D
:101450009C2D0E94F109DF91CF911F910F91FF9078
:10146000EF90DF90CF90BF9008950F931F93CF938D
:10147000DF93EC01162F042F60E0413009F461E0A6
:101480008B850E94280D8C858F3F19F060E00E94AB
:10149000280D023091F08C8184FF04C0CE01612FB1
:1014A00048E00EC0612F70E084E0759567958A95DD
:1014B000E1F7CE0144E00E94010ACE01612F44E031
:1014C0000E94010ADF91CF911F910F9108956F92B1
:1014D0007F928F92AF92CF92EF920F931F93DF93F1
:1014E000CF93CDB7DEB73C01162F8E2DF301438786
:1014F00024870587E686C786A08A818A9D85928B88
:101500009E85938B9F85948B9889958B61E00E9433
:10151000E90CF301878561E00E94E90CF301808901
:1015200061E00E94E90CF301818961E00E94E90C0D
:101530001123A1F4F301828961E00E94E90CF30117
:10154000838961E00E94E90CF301848961E00E94D3
:10155000E90CF301858961E00E94E90CF3018385C0
:1015600061E00E94E90CF30184858F3F19F061E08E
:101570000E94E90CF301858561E00E94E90C1123CA
:1015800019F0F301148203C080E1F3018483F301B5
:10159000838560E00E94280DF301858560E00E944C
:1015A000280DF30184858F3F19F060E00E94280D1B
:1015B0008FEFF301868B12861186CF91DF911F91F9
:1015C0000F91EF90CF90AF908F907F906F90089594
:1015D000DF92EF92FF920F931F938C01D62E7A0128
:1015E000862F61E00E94E90CD8015696DC9256974E
:1015F0001A96FC92EE921997ED91FC910084F18578
:10160000E02DC80160E009951F910F91FF90EF90C8
:10161000DF900895DC01362F56962C9156972F3F78
:1016200061F1E22FF0E0E255FF4FE491EE2389F003
:1016300019968D919C911A97892B19F4822F70E03D
:1016400005C06FEF70E0631B7109822F0E94890C47
:10165000089519968D919C911A97662319F0892BFC
:1016600041F402C0019729F4822F61E00E94280D05
:101670000895822F60E00E94280D08956F927F9256
:101680008F92AF92BF92CF92DF92EF92FF920F9321
:101690001F933C01162FF42ED22EB02EAE2C8C2C84
:1016A0000E94D1088AE592E0D3018D939C9300D0EB
:1016B00000D0EDB7FEB73196ADB7BEB711961C920C
:1016C000118212821382C30161E0412F2FEF0F2D8F
:1016D000ED2CCB2C0E94670A0F900F900F900F906B
:1016E0001F910F91FF90EF90DF90CF90BF90AF9040
:1016F0008F907F906F9008951F920F920FB60F9268
:1017000011242F933F934F935F936F937F938F9306
:101710009F93AF93BF93EF93FF93E091CA02F09131
:10172000CB020995FF91EF91BF91AF919F918F915E
:101730007F916F915F914F913F912F910F900FBECD
:101740000F901F9018951F920F920FB60F921124B1
:101750002F933F938F939F93AF93BF938091D0022A
:101760009091D102A091D202B091D3023091D402D3
:101770000196A11DB11D232F2D5F2D3720F02D5770
:101780000196A11DB11D2093D4028093D0029093A5
:10179000D102A093D202B093D3028091CC02909157
:1017A000CD02A091CE02B091CF020196A11DB11D34
:1017B0008093CC029093CD02A093CE02B093CF023F
:1017C000BF91AF919F918F913F912F910F900FBE3D
:1017D0000F901F9018959B01AC017FB7F8948091F2
:1017E000CC029091CD02A091CE02B091CF0266B50D
:1017F000A89B05C06F3F19F00196A11DB11D7FBFC9
:10180000BA2FA92F982F8827860F911DA11DB11DD2
:1018100062E0880F991FAA1FBB1F6A95D1F7BC0110
:101820002DC0FFB7F8948091CC029091CD02A09189
:10183000CE02B091CF02E6B5A89B05C0EF3F19F0EC
:101840000196A11DB11DFFBFBA2FA92F982F882780
:101850008E0F911DA11DB11DE2E0880F991FAA1FD7
:10186000BB1FEA95D1F7861B970B885E9340C8F2A1
:10187000215030404040504068517C4F2115310587
:101880004105510571F60895019739F0880F991FA8
:10189000880F991F02970197F1F70895789484B5FE
:1018A000826084BD84B5816084BD85B5826085BD5C
:1018B00085B5816085BDEEE6F0E080818160808342
:1018C000E1E8F0E010828081826080838081816025
:1018D0008083E0E8F0E0808181608083E1EBF0E0EC
:1018E000808184608083E0EBF0E080818160808390
:1018F000EAE7F0E080818460808380818260808379
:101900008081816080838081806880831092C100A3
:1019100008951F93CF93DF93182FEB0161E00E948E
:10192000E90C209709F44AC0CF3FD10509F449C01A
:10193000E12FF0E0E255FF4F84918330C1F0843015
:1019400028F4813051F08230B1F50CC0863019F1A5
:10195000873049F1843079F514C084B5806884BD3E
:10196000C7BD33C084B5806284BDC8BD2EC0809120
:101970008000806880938000D0938900C0938800A5
:1019800024C080918000806280938000D0938B007F
:10199000C0938A001AC08091B00080688093B00024
:1019A000C093B30012C08091B00080628093B000F9
:1019B000C093B4000AC0C038D1051CF4812F60E088
:1019C00002C0812F61E00E94280DDF91CF911F910D
:1019D0000895CF93DF93482F50E0CA0186569F4F5A
:1019E000FC0134914A575F4FFA018491882369F1D1
:1019F00090E0880F991FFC01E859FF4FA591B49121
:101A0000FC01EE58FF4FC591D491662351F42FB7D6
:101A1000F8948C91932F909589238C9388818923B6
:101A20000BC0623061F42FB7F8948C91932F90958E
:101A300089238C938881832B88832FBF06C09FB70F
:101A4000F8948C91832B8C939FBFDF91CF91089555
:101A5000482F50E0CA0182559F4FFC012491CA01D2
:101A600086569F4FFC0194914A575F4FFA0134917B
:101A7000332309F440C0222351F1233071F0243084
:101A800028F42130A1F0223011F514C02630B1F035
:101A90002730C1F02430D9F404C0809180008F77C2
:101AA00003C0809180008F7D8093800010C084B53A
:101AB0008F7702C084B58F7D84BD09C08091B0004E
:101AC0008F7703C08091B0008F7D8093B000E32FAB
:101AD000F0E0EE0FFF1FEE58FF4FA591B4912FB726
:101AE000F894662321F48C919095892302C08C91FF
:101AF000892B8C932FBF0895682F70E0CB018255FE
:101B00009F4FFC012491CB0186569F4FFC014491CD
:101B10006A577F4FFB019491992319F420E030E03C
:101B20003CC0222351F1233071F0243028F42130BD
:101B3000A1F0223011F514C02630B1F02730C1F0E9
:101B40002430D9F404C0809180008F7703C0809145
:101B500080008F7D8093800010C084B58F7702C095
:101B600084B58F7D84BD09C08091B0008F7703C09C
:101B70008091B0008F7D8093B000892F90E0880F16
:101B8000991F84589F4FFC01A591B4918C9120E03E
:101B900030E0842311F021E030E0C90108958F92F4
:101BA0009F92AF92BF92CF92DF92EF92FF920F93EC
:101BB0001F93CF93DF93A82FB0E0CD0186569F4FA0
:101BC000FC018490AA57BF4FFD018491662311F454
:101BD000992401C0982C6FEFA62E6FEFB62E6FEFF1
:101BE000C62E6FE0D62EA222B322C422D522682FA1
:101BF00070E0660F771F64587F4FEE24FF24870143
:101C0000FB01A591B4910BC0EA14FB040C051D0562
:101C100009F44EC00894E11CF11C011D111D8C91AA
:101C20008821891589F30CC0EA14FB040C051D05F5
:101C300009F43EC00894E11CF11C011D111D03C0F4
:101C4000FB01A591B4918C918821891569F720E059
:101C500030E040E050E0FB01C591D4910FC0DA01C3
:101C6000C9018E0D9F1DA01FB11F8A159B05AC05D4
:101C7000BD05F1F02F5F3F4F4F4F5F4F88818821A7
:101C8000891569F3CA01B90125E130E040E050E06F
:101C90000E9489129B01AC01205F3F4F4F4F5F4F65
:101CA00084E056954795379527958A95D1F704C0D6
:101CB00020E030E040E050E0B901CA01DF91CF916F
:101CC0001F910F91FF90EF90DF90CF90BF90AF905A
:101CD0009F908F900895CF93DF930E944E0C0E94A7
:101CE0006106C0E0D0E00E94C5072097E1F30E94A2
:101CF0000000F9CF08950E94860F0895CF92DF92D9
:101D0000EF92FF920F931F93CF93DF937C016B01B0
:101D10008A01C0E0D0E00FC0D6016D916D01D701FE
:101D2000ED91FC910190F081E02DC7010995C80F5C
:101D3000D91F015010400115110571F7CE01DF9137
:101D4000CF911F910F91FF90EF90DF90CF9008956A
:101D5000DC01ED91FC910190F081E02D0995089551
:101D6000CF93DF93EC016115710519F420E030E0A9
:101D70000FC0DB010D900020E9F71197A61BB70BF0
:101D8000E881F9810280F381E02DAD0109959C0184
:101D9000C901DF91CF9108954F925F927F928F9208
:101DA0009F92AF92BF92CF92DF92EF92FF920F93EA
:101DB0001F93DF93CF93CDB7DEB7A1970FB6F894FB
:101DC000DEBF0FBECDBF2C01742ECB01223008F434
:101DD0002AE019A231E2C32ED12CCC0EDD1E822EB8
:101DE0009924AA24BB24672D752FA50194010E9474
:101DF000A81279018A01C801B701A50194010E94C6
:101E00008912472D461B0894C108D1084A3014F4A2
:101E1000405D01C0495CF6014083E114F104010515
:101E2000110521F07E2C5F2DC801DDCFC201B60166
:101E30000E94B00EA1960FB6F894DEBF0FBECDBFC4
:101E4000CF91DF911F910F91FF90EF90DF90CF9096
:101E5000BF90AF909F908F907F905F904F9008952C
:101E6000CF92DF92EF92FF920F931F93CF93DF9366
:101E7000EC016A017B012115310541F4E881F9810A
:101E80000190F081E02D642F09951FC02A303105A3
:101E9000D1F477FF17C0E881F9810190F081E02D3E
:101EA0006DE209958C0144275527BA014C195D094B
:101EB0006E097F09CE012AE00E94CC0E9801280FFE
:101EC000391F04C02AE00E94CC0E9C01C901DF9199
:101ED000CF911F910F91FF90EF90DF90CF900895D9
:101EE000EF92FF920F931F937B019A010027F7FC5B
:101EF0000095102FB801A7010E94300F1F910F917C
:101F0000FF90EF9008950E94B00E08950F931F93D5
:101F1000CF93DF93BC018230910510F462E070E052
:101F2000E091D502F091D602A0E0B0E040E050E0B0
:101F300024C08081918186179707D0F08617970774
:101F400071F482819381109729F013969C938E935C
:101F500012972CC09093D6028093D50227C04115CA
:101F6000510519F08417950718F4EF018D01AC01A4
:101F7000DF01828193819C01F9013097D1F64115EF
:101F80005105F9F0CA01861B970B8430910580F446
:101F90008A819B810115110521F0F80193838283C9
:101FA00004C09093D6028093D502FE0132962FC0D2
:101FB000FE01E80FF91F619371930297998388835B
:101FC00026C08DB79EB78857904020913A02309135
:101FD0003B0228173907C8F4AC01421B530B4617C4
:101FE000570798F0CB0102964817590770F0820FF7
:101FF000931F90933B0280933A0290933D0280930B
:102000003C02F9016193719302C0E0E0F0E0CF017E
:10201000DF91CF911F910F9108955058BB27AA27A8
:102020000ED075C166D130F06BD120F031F49F3FF6
:1020300011F41EF45BC10EF4E095E7FB51C1E92FEA
:1020400077D180F3BA17620773078407950718F0F2
:1020500071F49EF58FC10EF4E0950B2EBA2FA02DD2
:102060000B01B90190010C01CA01A0011124FF2745
:10207000591B99F0593F50F4503E68F11A16F04040
:10208000A22F232F342F4427585FF3CF469537953F
:102090002795A795F0405395C9F77EF41F16BA0B04
:1020A000620B730B840BBAF09150A1F0FF0FBB1FB2
:1020B000661F771F881FC2F70EC0BA0F621F731FFB
:1020C000841F48F4879577956795B795F7959E3F58
:1020D00008F0B3CF9395880F08F09927EE0F9795E6
:1020E00087950895D9D008F481E008950CD00FC1E8
:1020F00007D140F0FED030F021F45F3F19F0F0C07E
:10210000511139C1F3C014D198F39923C9F3552360
:10211000B1F3951B550BBB27AA27621773078407DA
:1021200038F09F5F5F4F220F331F441FAA1FA9F390
:1021300033D00E2E3AF0E0E830D091505040E69582
:10214000001CCAF729D0FE2F27D0660F771F881FE3
:10215000BB1F261737074807AB07B0E809F0BB0BD2
:10216000802DBF01FF2793585F4F2AF09E3F5105F6
:1021700068F0B6C000C15F3FECF3983EDCF3869593
:1021800077956795B795F7959F5FC9F7880F911D6C
:102190009695879597F90895E1E0660F771F881F58
:1021A000BB1F621773078407BA0720F0621B730B0B
:1021B000840BBA0BEE1F88F7E095089504D068945D
:1021C000B111D9C00895BCD088F09F5790F0B92FB5
:1021D0009927B751A0F0D1F0660F771F881F991F7C
:1021E0001AF0BA95C9F712C0B13081F0C3D0B1E08E
:1021F0000895C0C0672F782F8827B85F39F0B93F9E
:10220000CCF3869577956795B395D9F73EF490957D
:102210008095709561957F4F8F4F9F4F0895E894FB
:1022200009C097FB3EF490958095709561957F4F1E
:102230008F4F9F4F9923A9F0F92F96E9BB279395CC
:10224000F695879577956795B795F111F8CFFAF4DC
:10225000BB0F11F460FF1BC06F5F7F4F8F4F9F4F0D
:1022600016C0882311F096E911C0772321F09EE86B
:10227000872F762F05C0662371F096E8862F70E0D1
:1022800060E02AF09A95660F771F881FDAF7880FAB
:102290009695879597F90895990F0008550FAA0B01
:1022A000E0E8FEEF16161706E807F907C0F0121669
:1022B0001306E407F50798F0621B730B840B950B6C
:1022C00039F40A2661F0232B242B252B21F40895C1
:1022D0000A2609F4A140A6958FEF811D811D08955E
:1022E00097F99F6780E870E060E008959FEF80ECC9
:1022F000089500240A94161617061806090608956C
:1023000000240A9412161306140605060895092ED1
:102310000394000C11F4882352F0BB0F40F4BF2B40
:1023200011F460FF04C06F5F7F4F8F4F9F4F089580
:1023300057FD9058440F551F59F05F3F71F0479576
:10234000880F97FB991F61F09F3F79F0879508955B
:10235000121613061406551FF2CF4695F1DF08C07A
:10236000161617061806991FF1CF86957105610597
:1023700008940895E894BB2766277727CB0197F93F
:1023800008950BD0C4CFB5DF28F0BADF18F095233D
:1023900009F0A6CFABCF1124EECFCADFA0F3959FF3
:1023A000D1F3950F50E0551F629FF001729FBB273C
:1023B000F00DB11D639FAA27F00DB11DAA1F649FE8
:1023C0006627B00DA11D661F829F2227B00DA11D9B
:1023D000621F739FB00DA11D621F839FA00D611D21
:1023E000221F749F3327A00D611D231F849F600D42
:1023F000211D822F762F6A2F11249F5750408AF07B
:10240000E1F088234AF0EE0FFF1FBB1F661F771F06
:10241000881F91505040A9F79E3F510570F060CF42
:10242000AACF5F3FECF3983EDCF3869577956795EE
:10243000B795F795E7959F5FC1F7FE2B880F911D24
:102440009695879597F9089511F40EF44FCF4AC0E9
:1024500077DFD0F39923D9F3CEF39F57550B87FF3E
:1024600051D056959795B0E020F4660F771F881FDE
:10247000BB1F1F930F9300249001A0018001F00166
:10248000A0E80E0F1F1F0A1E511D601B710B800953
:10249000B50B48F4600F711F801DB51F0E1B1F0B7D
:1024A0000A0A510907C02E0F3F1F4A1F0E0F1F1F98
:1024B0000A1E511D660F771F881FBB1FA695F79533
:1024C000E795F8F60617170708065B07211D311D6B
:1024D000411D0F911F91B901842F9158880F969536
:1024E000879508959F3F49F0915028F486957795F8
:1024F0006795B7959F5F80389F4F880F9695879512
:1025000097F9089591505040660F771F881FD2F7B2
:102510000895629FD001739FF001829FE00DF11D2D
:10252000649FE00DF11D929FF00D839FF00D749F4D
:10253000F00D659FF00D9927729FB00DE11DF91FF9
:10254000639FB00DE11DF91FBD01CF011124089556
:10255000A1E21A2EAA1BBB1BFD010DC0AA1FBB1FA7
:10256000EE1FFF1FA217B307E407F50720F0A21B19
:10257000B30BE40BF50B661F771F881F991F1A9486
:1025800069F760957095809590959B01AC01BD01B0
:10259000CF01089597FB092E05260ED057FD04D0D4
:1025A000D7DF0AD0001C38F450954095309521951E
:1025B0003F4F4F4F5F4F0895F6F790958095709578
:1025C00061957F4F8F4F9F4F0895EE0FFF1F05902E
:0A25D000F491E02D0994F894FFCF78
:1025DA002020005900484D41204D4554504800489C
:1025EA000020202000202020202041004F005441BC
:1025FA000020202020202000202020204D45205986
:10260A0000455048584F5900202020200020202003
:10261A0020204D414E4F53204D41522E2020202044
:10262A0020002020202020323031342D3230313524
:10263A00202020202020005663633D2000205600E1
:10264A0054633D20002000430054663D20004600AC
:10265A0055733D2000206D2F73004820004B4559CB
:10266A0048200041200042480045490020454B418E
:10267A00544F0054412020202020200020494E544D
:10268A0000450020202020454B544F00204559503A
:10269A004F590020204D45545048004820410059C8
:1026AA004E415448202020005B315D203D204F4E92
:1026BA00202F20524553455420202020005B325DB4
:1026CA00203D204F4646202020000E1515150E04E9
:1026DA0004001515150E040404000E1111110E0044
:1026EA001F001F10101010101000040A11111111F0
:1026FA001F00040A1111111111001F1111111111DA
:10270A0011000E11111F1F1F1F00D70264000000C5
:10271A00000034097E0E7709CF08D0087A0E0040EF
:10272A001050004014540000000034097E0E77094E
:06273A00E80A0A0B350A53
:00000001FF
